:020000020000FC
:020000005EC0E0
:020018002BC2F9
:02003C001FC3E0
:0200800084C337
:0200B40026C460
:1000BC00CBC301E20EBF0FEF0DBF07E104B908E09F
:1000CC0005B901E00DBD00E50CBD289A2C980F9ADE
:1000DC0017980000179A0CE000936A0000E20DBB21
:1000EC00259A269A989AA09A2D982E982227992785
:1000FC00772789E250E000E0A02EB02E0BE200E959
:10010C000BE2A89500E004BF0EE10093600000E054
:10011C00009360000BEA009364000FE3009365000A
:10012C0000E900BF00E20093B60006E00093B100C6
:10013C000091B6000F71E1F707E00093170001E0A2
:10014C000093700040E883D12DD103EC289879D12D
:10015C00002777D1289A00EE289873D100E971D145
:10016C00289A01EE28986DD10BE26BD1289A02EEF9
:10017C00289867D103EC65D1289A03EE289861D1B1
:10018C0004EA5FD1289A08EC28985BD10BE259D18C
:10019C00289A05EC289855D100E853D1289A0CEEF2
:1001AC0028984FD108E34DD1289A0EEE289849D1C2
:1001BC0004E047D1289A0DEE289843D100E841D1AC
:1001CC00289A0FE828983DD1289A0EEC289839D116
:1001DC0008E037D1289AA8950EE10093600008E258
:1001EC00009360000FEF0CBB78942C9A07E003BFD0
:1001FC0065E088950000000000006A95D1F70027A3
:10020C0003BF2C9848E223D1D3D00CD126E030EA9E
:10021C004FEF1DD1863D49F13A95D1F7D2D020E070
:10022C00E4CFCFD020E055D200E00093A1000093A2
:10023C0072000000000000005230D9F300E000937F
:10024C0091000093210100938100009371000093B1
:10025C007300009380000BEA009364000FE300939B
:10026C0065002D982E9850E0C0CF03EA00936400EF
:10027C0007E00093650003EA0093800000E0009320
:10028C0089000093880000938B0000938A000AE099
:10029C000093810001D20000000000005130D9F31E
:1002AC0000E00093A5000093A40001E0009372000D
:1002BC0002E00093A1004AD3000000000FD0893265
:1002CC00D9F788270000000009D08932D9F7882790
:1002DC000000000003D08932D9F7A3CF7727929979
:1002EC0072E008D0103808F07160772311F0972B6A
:1002FC004CD008951127A09830E24FEFA8D03A9532
:10030C00E1F7A09A49E0A3D0A09849E0A0D0919938
:10031C001068A09A49E09BD0A09849E098D0919998
:10032C001064A09A49E093D0A09849E090D091999C
:10033C001062A09A49E08BD0A09849E088D091999E
:10034C001061A09A49E083D0A09849E080D091999F
:10035C001860A09A49E07BD0A09849E078D0919998
:10036C001460A09A49E073D0A09849E070D091999C
:10037C001260A09A49E06BD0A09849E068D091999E
:10038C001160A09A4FEF63D008951BD03CD0D8D009
:10039C0021E00000000000002530D9F712D042D037
:1003AC0026E0089502EC28984CD008E04AD0289A10
:1003BC0001E8289846D000E044D0289A0830C1F7CC
:1003CC00089502EC28983DD003E03BD0289A000019
:1003DC0000000000000001E8289833D000E031D084
:1003EC00289A083071F7089502EC28982AD009E071
:1003FC0028D0289A01E8289824D000E022D0289A06
:10040C000930C1F7089502EC28981BD009E119D0E6
:10041C00289A01E8289815D000E013D0289A0931C1
:10042C00C1F7089502EC28980CD006E10AD0289A5E
:10043C0001E8289806D000E004D0289A0631C1F7CC
:10044C0008950EBD0DB507FFFDCF0EB50895000044
:10045C0000000000000000000000000000004A95B1
:10046C00B1F708950F930FB70F930FE82898E9DFB2
:10047C00289A01E82898E5DF00E0E3DF289A0631A6
:10048C0029F1013119F10F31A1F3023191F302E895
:10049C002898D7DF00E0D5DF289A007E003600F0E0
:1004AC00213059F0223061F0233069F0243009F406
:1004BC0025E00F910FBF0F91189568D022E0F9CF6E
:1004CC008BD023E0F6CFAED024E0F3CF00E2289817
:1004DC00B8DF00E0B6DF003171F500E0B2DF00E01C
:1004EC00B0DF00E0AEDF003031F500E0AADF00E065
:1004FC00A8DF00E0A6DF00E0A4DF00E0A2DF043507
:10050C00D1F400E09EDF0B3BB1F400E09ADF002E4B
:10051C0000E097DF0B3A79F400E093DF063459F4EE
:10052C0000E08FDF073339F400E08BDF023D19F474
:10053C00802DAA24BB24289A0F910FBF0F911895D8
:10054C002C9A00002C9800E628987BDF00E179DFDC
:10055C0001E677DF08E875DF02E073DF03EC71DF9B
:10056C0004EA6FDF00EA6DDF0BE26BDF00E969DFA5
:10057C000BE267DF072F65DF07E663DF01EC61DF66
:10058C000AE85FDF0FE95DDF289A08952C9A0000D6
:10059C002C9800E6289855DF00E153DF01E651DF87
:1005AC0008E84FDF02E04DDF03EC4BDF04EA49DFE4
:1005BC0000EB47DF0BE245DF00E943DF0BE241DFF5
:1005CC00072F3FDF07E63DDF01EC3BDF0AE839DFB1
:1005DC000FE937DF289A08952C9A00002C9800E632
:1005EC0028982FDF00E12DDF01E62BDF08E829DF5B
:1005FC0002E027DF03EC25DF04EA23DF00EC21DF38
:10060C000BE21FDF00E91DDF0BE21BDF072F19DFF9
:10061C0007E617DF01EC15DF0AE813DF0FE911DF3E
:10062C00289A08952C9A00002C9800E6289809DF47
:10063C0000E107DF01E605DF08E803DF02E001DF88
:10064C0003ECFFDE04EAFDDE00EDFBDE0BE2F9DE7F
:10065C0000E9F7DE0BE2F5DE072FF3DE07E6F1DE4D
:10066C0001ECEFDE0AE8EDDE0FE9EBDE289A0895E7
:10067C000000000000000F930FB70F9301E0A00ED5
:10068C000027B01E28F0A8950F910FBF0F91189559
:10069C00000000000000FCCF00E0009395000093E8
:1006AC0094000EE40093990000E20093980002E09D
:1006BC000093710005E0009391000FEF0093890007
:1006CC000093880000E000938B0000938A0051E0B7
:1006DC00089500E000932501009324010EE400939B
:1006EC00290100E20093280102E00093730005E069
:1006FC00009321010FEF00938B0000938A0000E020
:10070C00009389000093880052E008955330B9F0AB
:10071C005430A9F000E0009395000093940001E0A0
:10072C000093990000E00093980002E000937100A0
:10073C000AE000939100B0E2AA27D4E2CC2753E060
:10074C0008955530D1F05630C1F000E000932501EA
:10075C000093240102E00093290100E0009328019A
:10076C0002E0009373000AE0009321010FE3009371
:10077C008B0000938A00D0E2CC2755E008950F93AC
:10078C000FB70F93513069F05330C9F05430B9F0B2
:10079C0000E000939100009371000F910FBF0F9137
:1007AC00189500E00093910000937100009389006C
:1007BC000093880050E00F910FBF0F911895FE0128
:1007CC0005901590F772400103EBCDD0EF0190929C
:1007DC008B0080928A00FD0105901590400103EB7F
:1007EC00C2D0DF01F83241F09092890080928800EB
:1007FC000F910FBF0F911895543051F0B0E2AA270A
:10080C0090928900809288000F910FBF0F911895DC
:10081C0000E0009391000093710000938900009315
:10082C00880000938B0000938A00042D013039F06E
:10083C00033029F08BD00F910FBF0F91189581DFEA
:10084C000F910FBF0F9118950F930FB70F93523055
:10085C0069F05530C9F05630B9F000E00093210131
:10086C00009373000F910FBF0F91189500E0009348
:10087C0021010093730000938B0000938A0050E0D9
:10088C000F910FBF0F911895FE0105901590400127
:10089C0000E869D0EF01F83241F090928900809223
:1008AC0088000F910FBF0F911895563051F0D0E280
:1008BC00CC2790928900809288000F910FBF0F91E6
:1008CC00189500E0009321010093730000938900B8
:1008DC000093880000938B0000938A00042D023053
:1008EC0029F034D00F910FBF0F9118950FDF0F9196
:1008FC000FBF0F9118950F930FB70F93903061F0B6
:10090C00913099F09230B9F0933079F0492E9927C3
:10091C000F910FBF0F911895533019F0553019F0F6
:10092C00F5CF54E0F3CF56E0F1CF5330D1F3543040
:10093C00C1F307DFEBCF5530B1F35630A1F3E6DE50
:10094C00E5CF54E0E3CFE2DEFCDEE0CF02E0009343
:10095C0089000CEC0093880000E000938B0000935E
:10096C008A0057E00895909E1001809E0027210C6C
:06097C00301E4101089548
:1020000000000000000000000000000000000000D0
:1020100001000100010001000100020002000200B5
:102020000200030003000300040004000500050093
:102030000600060006000700080008000900090065
:102040000A000A000B000C000C000D000E000F002F
:102050000F001000110012001300130014001500EF
:1020600016001700180019001A001B001C001D00A4
:102070001E001F0020002100220023002500260052
:102080002700280029002B002C002D002E003000F6
:1020900031003200340035003700380039003B0091
:1020A0003C003E003F004100420044004600470023
:1020B00049004A004C004E004F00510053005400AC
:1020C000560058005A005B005D005F00610063002D
:1020D0006500660068006A006C006E0070007200A7
:1020E0007400760078007A007C007E008000820018
:1020F0008400860089008B008D008F009100930082
:10210000960098009A009C009F00A100A300A600E2
:10211000A800AA00AD00AF00B100B400B600B8003E
:10212000BB00BD00C000C200C500C700CA00CC0093
:10213000CF00D100D400D600D900DB00DE00E100E2
:10214000E300E600E800EB00EE00F000F300F6002C
:10215000F800FB00FE0000010301060109010B016C
:102160000E0111011401160119011C011F012201A8
:10217000250127012A012D013001330136013901E2
:102180003B013E014101440147014A014D0150011B
:102190005301560159015C015F016201650168014B
:1021A0006B016E017101740177017A017D0180017B
:1021B0008301860189018C018F01920195019801AB
:1021C0009B019E01A101A501A801AB01AE01B101D6
:1021D000B401B701BA01BD01C001C401C701CA0100
:1021E000CD01D001D301D601D901DD01E001E30128
:1021F000E601E901EC01EF01F201F601F901FC0150
:10220000FF010202050208020C020F02120215026F
:1022100018021B021E022102250228022B022E0296
:102220003102340237023A023E02410244024702BE
:102230004A024D0250025302560259025D026002E8
:102240006302660269026C026F0272027502780212
:102250007B027E028102840287028A028D02900242
:102260009302960299029C029F02A202A502A80272
:10227000AB02AE02B102B402B702BA02BD02C002A2
:10228000C302C502C802CB02CE02D102D402D702D9
:10229000D902DC02DF02E202E502E802EA02ED0214
:1022A000F002F302F502F802FB02FE020003030350
:1022B000060308030B030E0310031303160318038E
:1022C0001B031D0320032303250328032A032D03D7
:1022D0002F0332033403370339033C033E03410326
:1022E0004303460348034A034D034F03510354037A
:1022F000560358035B035D035F03620364036603D5
:1023000068036B036D036F03710373037503780335
:102310007A037C037E03800382038403860388039D
:102320008A038C038E03900392039403960398030D
:1023300099039B039D039F03A103A303A403A60387
:10234000A803AA03AB03AD03AF03B003B203B40306
:10235000B503B703B803BA03BC03BD03BF03C0038F
:10236000C203C303C503C603C703C903CA03CC031F
:10237000CD03CE03D003D103D203D303D503D603B9
:10238000D703D803D903DB03DC03DD03DE03DF035C
:10239000E003E103E203E303E403E503E603E70309
:1023A000E803E903EA03EB03EB03EC03ED03EE03BD
:1023B000EF03EF03F003F103F203F203F303F4037B
:1023C000F403F503F503F603F603F703F803F80344
:1023D000F803F903F903FA03FA03FB03FB03FB0316
:1023E000FC03FC03FC03FC03FD03FD03FD03FD03F1
:1023F000FD03FE03FE03FE03FE03FE03FE03FE03D6
:10240000FE03FE03FE03FE03FE03FE03FE03FE03C4
:10241000FD03FD03FD03FD03FD03FC03FC03FC03BF
:10242000FC03FB03FB03FB03FA03FA03F903F903C1
:10243000F803F803F803F703F603F603F503F503CF
:10244000F403F403F303F203F203F103F003EF03E5
:10245000EF03EE03ED03EC03EB03EB03EA03E90305
:10246000E803E703E603E503E403E303E203E10330
:10247000E003DF03DE03DD03DC03DB03D903D80362
:10248000D703D603D503D303D203D103D003CE039E
:10249000CD03CC03CA03C903C703C603C503C303E3
:1024A000C203C003BF03BD03BC03BA03B803B70331
:1024B000B503B403B203B003AF03AD03AB03AA0388
:1024C000A803A603A403A303A1039F039D039B03E7
:1024D0009903980396039403920390038E038C034D
:1024E0008A03880386038403820380037E037C03BC
:1024F0007A0378037503730371036F036D036B0332
:1025000068036603640362035F035D035B035803B0
:102510005603540351034F034D034A034803460334
:10252000430341033E033C033903370334033203BF
:102530002F032D032A0328032503230320031D0350
:102540001B0318031603130310030E030B030803E6
:10255000060303030003FE02FB02F802F502F30286
:10256000F002ED02EA02E802E502E202DF02DC022A
:10257000D902D702D402D102CE02CB02C802C502D0
:10258000C302C002BD02BA02B702B402B102AE0277
:10259000AB02A802A502A2029F029C029902960227
:1025A000930290028D028A028702840281027E02D7
:1025B0007B027802750272026F026C026902660287
:1025C000630260025D0259025602530250024D023C
:1025D0004A024702440241023E023A0237023402F2
:1025E00031022E022B022802250221021E021B02AA
:1025F0001802150212020F020C0208020502020262
:10260000FF01FC01F901F601F201EF01EC01E90122
:10261000E601E301E001DD01D901D601D301D001DA
:10262000CD01CA01C701C401C001BD01BA01B70192
:10263000B401B101AE01AB01A801A501A1019E0148
:102640009B019801950192018F018C0189018601FE
:10265000830180017D017A017701740171016E01AE
:102660006B016801650162015F015C01590156015E
:10267000530150014D014A014701440141013E010E
:102680003B0139013601330130012D012A012701B7
:10269000250122011F011C0119011601140111015C
:1026A0000E010B010901060103010001FE00FB0000
:1026B000F800F600F300F000EE00EB00E800E600A2
:1026C000E300E000DE00DB00D900D600D400D1003A
:1026D000CF00CC00CA00C700C500C200C000BD00CA
:1026E000BB00B800B600B400B100AF00AD00AA0056
:1026F000A800A600A300A1009F009C009A009800DB
:102700009600930091008F008D008B008900860059
:102710008400820080007E007C007A0078007600D1
:102720007400720070006E006C006A006800660041
:102730006500630061005F005D005B005A005800A7
:1027400056005400530051004F004E004C004A0008
:102750004900470046004400420041003F003E005F
:102760003C003B00390038003700350034003200AF
:10277000310030002E002D002C002B0029002800F5
:1027800027002600250023002200210020001F0032
:102790001E001D001C001B001A0019001800170065
:1027A0001600150014001300130012001100100091
:1027B0000F000F000E000D000C000C000B000A00B3
:1027C0000A000900090008000800070006000600CA
:1027D00006000500050004000400030003000300D8
:1027E00002000200020002000100010001000100DD
:1027F00001000000000000000000000000000000D8
:00000001FF
